S01D000062696E2F6F70656E626C745F73746D3332663330332E7372656397
S3150800000000300020590200089F020008A1020008DB
S31508000010A3020008A5020008A702000800000000C5
S31508000020000000000000000000000000A90200080F
S31508000030AB02000800000000AD020008D51C00084D
S31508000040B1020008B3020008B5020008B7020008AA
S31508000050B9020008BB020008BD020008BF0200087A
S31508000060C1020008C3020008C5020008C70200084A
S31508000070C9020008CB020008CD020008CF0200081A
S31508000080D1020008D3020008D5020008D7020008EA
S31508000090D9020008DB020008DD020008DF020008BA
S315080000A0E1020008E3020008E5020008E70200088A
S315080000B0E9020008EB02000800000000ED02000853
S315080000C0EF0200080000000000000000F10200082E
S315080000D000000000F3020008F5020008F702000815
S315080000E0F9020008FB0200080000000000000000FA
S315080000F000000000000000000000000000000000F2
S3150800010000000000000000000000000000000000E1
S315080001100000000000000000FD020008FF020008C1
S3150800012000000000000000000000000000000000C1
S3150800013000000000000000000000000000000000B1
S315080001400103000803030008000000000000000087
S315080001500000000000000000000000000000000091
S315080001600000000000000000000000000000000081
S315080001700000000000000000000000000000000071
S31508000180000000000503000810B5054C237833B9B4
S31508000190044B13B10448AFF300800123237010BD4C
S315080001A07000002000000000341E0008084B10B53F
S315080001B01BB108490848AFF300800848036803B92B
S315080001C010BD074B002BFBD0BDE81040184700BFF9
S315080001D00000000074000020341E00087000002093
S315080001E000000000154B002B08BF134B9D46A3F5D6
S315080001F0803A00218B460F461348144A121A01F01A
S31508000200B5FD0F4B002B00D098470E4B002B00D0A6
S3150800021098470020002104000D000D48002802D050
S315080002200C48AFF3008001F07BFD2000290000F0A8
S315080002306FF801F061FD00BF0000080000300020E3
S3150800024000000000000000007000002020060020CA
S3150800025000000000000000000649074A074B9A42C2
S31508000260BEBF51F8040B42F8040BF8E70448804770
S3150800027004480047401E00080000002070000020C7
S3150800028069050008E50100081F49204A002301E026
S3150800029041F8043B9142FBD300F03AF8FEE7FEE74B
S315080002A0FEE7FEE7FEE7FEE7FEE7FEE7FEE7FEE718
S315080002B0FEE7FEE7FEE7FEE7FEE7FEE7FEE7FEE708
S315080002C0FEE7FEE7FEE7FEE7FEE7FEE7FEE7FEE7F8
S315080002D0FEE7FEE7FEE7FEE7FEE7FEE7FEE7FEE7E8
S315080002E0FEE7FEE7FEE7FEE7FEE7FEE7FEE7FEE7D8
S315080002F0FEE7FEE7FEE7FEE7FEE7FEE7FEE7FEE7C8
S31508000300FEE7FEE7FEE7000070000020200600205A
S3150800031008B500F0D9FF294A136823F0070343F00C
S3150800032002031360136803F00703022B03D06A2144
S31508000330234801F085F9234A136843F00103136043
S315080003401168204B8807FBD5196821F0F80141F0A0
S3150800035080011960596821F4741141F460115960DB
S31508000360D96A21F00F01D962196841F080711960C4
S315080003701168144B8901FBD5596821F0F0015960C1
S31508000380596821F4E06141F480615960596821F4A3
S3150800039060515960596821F0030141F00201596022
S315080003A0536803F00C03082BFAD1074800F06CF9E0
S315080003B001F028F901F035F9FCE700BF00200240FA
S315080003C0941D0008001002400090D003F0B5334B8E
S315080003D0334E9A6942F001029A619A698DB002F029
S315080003E001020592059A5A6942F400325A615A691D
S315080003F002F400320492049A5A6942F480225A613D
S315080004005A6902F480220392039ADA6942F40032A6
S31508000410DA61DA6902F400320292029ADA6942F083
S315080004200072DA61DB6903F0007300240125019389
S31508000430082706A93046019B06970795089409944C
S315080004400A9400F015FDB7624FF4007306A94FF041
S315080004509040069307940A9500F00AFD48F20403B3
S31508000460069302270326072306A94FF090400B930D
S315080004700797089609940A9500F0FAFC4FF4C053BA
S31508000480069306A909234FF0904007970896099402
S315080004900A940B9300F0ECFC0DB0F0BD001002407E
S315080004A0000400480F4808B50823836200F08AFC58
S315080004B04FF0904000F086FC0B4BDA6922F0007290
S315080004C0DA61DA6922F40032DA615A6922F48022A2
S315080004D05A615A6922F400325A619A6922F0010275
S315080004E09A6108BD000400480010024008B500F0F3
S315080004F035F84FF090431869C0F3402008BD6420D2
S3150800050000F002B800F006B8014B1880704700BF2B
S315080005109000002010B501F0CDFB0C4B1A689042F4
S315080005201C4611D30A4B0B4A1878082118B9012022
S315080005301870916102E000201870916201F0BAFB10
S31508000540054B1B881844206010BD00BF8C00002096
S31508000550920000200004004890000020014B082269
S315080005609A627047000400481549D1F8883043F468
S315080005707003C1F88830134B1A6842F001021A60FA
S315080005805868114A02405A601A6822F0847222F4A6
S3150800059080321A601A6822F480221A605A6822F495
S315080005A0FE025A60DA6A22F00F02DA62186B074A0C
S315080005B002401A6300229A604FF000638B6070470E
S315080005C000ED00E0001002400CC07FF8CCFC00FFF4
S315080005D0FEE7000030B50446006810F0010085B05B
S315080005E00D4601D0002045E0EB686A6821681A4389
S315080005F02B691A43AB691A431F4B0B4013432360FD
S31508000600636823F44052AB6813436360A36823F41A
S3150800061040726B691343A360184B9C4202D100F0E9
S31508000620FFFD0BE0164B9C4204D1684600F0E8FD3E
S31508000630029803E0134B9C42D4D1F6E70028D1D0A8
S315080006402A68002ACED0AB69B3F5004F4FEA5203A9
S315080006500AD103EB40004FF6F073B0FBF2F003400B
S31508000660C0F34200184303E01844B0FBF2F080B22E
S31508000670E060012005B030BDF369FFEF00380140A6
S315080006800044004000480040014B1860704700BF16
S3150800069000000020F0B504684B69012202FA03F352
S315080006A0D4F8002242F00102C4F800220568D5F801
S315080006B01C22DC432240C5F81C22CA69C2B9056857
S315080006C0D5F80C222240C5F80C224A69CF688D88D5
S315080006D00668483245EA074546F832504E690268C8
S315080006E08F680D88483602EBC60245EA074555600D
S315080006F0CA69012A18D10568D5F80C221A43C5F823
S315080007000C224A690F688D880668483245EA07450B
S3150800071046F832504E6902688F688D89483602EB72
S31508000720C60245EA074555608D6902681DB9D2F8C3
S315080007300452254002E0D2F804521D43C2F804527E
S315080007400D6902681DB9D2F814522C4002E0D2F89D
S3150800075014421C43C2F814420A6A012A01BF0168FE
S31508000760D1F81C221343C1F81C320268D2F80032B1
S3150800077023F00103C2F800320020F0BD704770B5BF
S315080007800446002800F0978090F83D3003F0FF02F9
S315080007901BB980F83C20FFF7F1FF2268022384F892
S315080007A03D30136823F0020313602268136843F090
S315080007B00103136001F086FA064623685A6812F0A8
S315080007C001050AD101F07EFA801B0A28F5D9032013
S315080007D084F83D0084F83C5070BD5A68D10767D547
S315080007E0A269012A1A680CBF42F0800222F0800230
S315080007F01A60E369012B23681A680CBF42F04002AD
S3150800080022F040021A60236A012B23681A680CBF7B
S3150800081042F0200222F020021A60636A012B236844
S315080008201A680CBF42F0100222F010021A60A36A7E
S31508000830012B23681A680CBF42F0080222F008024E
S315080008401A60E36A012B23681A680CBF42F0040297
S3150800085022F004021A60E368A26821681A43236931
S315080008601A4363691A436368013B1343CB612268E1
S31508000870136823F00103136001F024FA0546236880
S315080008805A68D2070BD501F01DFA401B0A28F6D97B
S315080008900320002384F83D0084F83C3070BD586876
S315080008A010F0010004D10123206484F83D3070BDA6
S315080008B0042384F83D30012070BD00002DE9F8437B
S315080008C0026893685B0104460E4606D493681F01C6
S315080008D003D49368D80040F1C38094F83C30012BC8
S315080008E000F0C480012384F83C3094F83D30DBB234
S315080008F0322B05D0622B05D0222B05D1422304E0EA
S31508000900522302E0722300E0122384F83D309368F4
S31508000910590106D4936813F0006F14BF0125022508
S3150800092000E000252B011A44D2F8801101F00101DC
S31508000930C2F88011206B2168D0F808E0C268194413
S31508000940D1F88071BEF1000F04D100683A4342EA3B
S31508000950405205E04EEA070740683A4342EAC002B9
S31508000960C1F88021216BDFF814810A69DFF8089144
S3150800097002F00F020A6122681A44D2F8841121F0A3
S315080009800F01C2F884112268216B1A440969D2F84A
S3150800099084010143C2F884112268216B1A4449690B
S315080009A0C2F888112268216B1A448969C2F88C1129
S315080009B022681344D3F8802142F00102C3F880214B
S315080009C001F080F907462B4A236899681DB9294B17
S315080009D00B409B1A0AE0012D04D1274B0B40B3EBC1
S315080009E0090303E0254B0B40B3EB080318BF0123AB
S315080009F0FBB1731CE8D046B9032384F83D3023685D
S31508000A004DB99A6842F080020CE001F05BF9C01B10
S31508000A108642D8D2F0E79A68012D0CBF42F400420C
S31508000A2042F400029A60002384F83C300320BDE8B3
S31508000A30F88394F83D30DBB2522B05D0722B05D0E3
S31508000A40422B05D1222304E0322302E0622300E090
S31508000A500123002084F83D3084F83C00BDE8F88383
S31508000A60042384F83D300120BDE8F8830220BDE860
S31508000A70F88300BF0100000400010008000001100F
S31508000A80F8B590F83C30012B04460D46164600F0A2
S31508000A90EB80012380F83C3099B990F83D30222B41
S31508000AA00BD090F83D30422B07D090F83D30622BA2
S31508000AB003D090F83D30722B16D1002384F83C30D1
S31508000AC0D2E001291CD190F83D30322BF5D090F8B0
S31508000AD03D30522BF1D090F83D30622BEDD090F896
S31508000AE03D30722B0CD1E8E790F83D30DBB2322B63
S31508000AF011D0522B11D0122B0CBF422322230FE008
S31508000B0094F83D30DBB2222B05D0422B05D0122BB0
S31508000B1005D1522304E0622302E0722300E0322367
S31508000B2084F83D3001F0CEF8074621680DB9CB6848
S31508000B3000E00B6913F0030F0CBF012300237BB100
S31508000B40731CF2D036B90320002384F83D0084F8DC
S31508000B503C30F8BD01F0B6F8C01B8642E5D2F2E794
S31508000B60626BA36B002D08BF134605F11B0210012B
S31508000B70095801F004019960266819B93158490DD8
S31508000B80196002E03158C90859602168120189586C
S31508000B90C1F34001D96021681144496801F00F0189
S31508000BA0196121680A4452681D62C2F30722DA6194
S31508000BB021682A011144D1F8B81119752168114420
S31508000BC0D1F8B811090A597521681144D1F8B81134
S31508000BD0090C997521681144D1F8B811090ED9750F
S31508000BE021681144D1F8BC11197621681144D1F84D
S31508000BF0BC11090A597621681144D1F8BC11090CAF
S31508000C00997621680A44D2F8BC21120EDA7623684E
S31508000C1065B9DA6842F02002DA6094F83D30DBB252
S31508000C20622B12D0722B12D0422B0BE01A6942F0BB
S31508000C3020021A6194F83D30DBB2622B09D0722B80
S31508000C4009D0522B09D1122308E0322306E0522399
S31508000C5004E0222302E0422300E00123002084F876
S31508000C603D3084F83C00F8BD0220F8BD0B4AD36835
S31508000C7013F0100305D00A49CB6943F00203CB6190
S31508000C801023D268520706D50549CA6942F00102FF
S31508000C90CA6143F00403014AD3607047002002404A
S31508000CA000060020064B1A69120641BF054A5A601B
S31508000CB002F1883200204CBF5A600120704700BFFD
S31508000CC00020024023016745034A136943F0800365
S31508000CD013610020704700BF0020024070B504462B
S31508000CE000F0F0FF114D0646EB6813F0010F0F4BAD
S31508000CF00AD0611CF8D00CB9032070BD00F0E2FFE1
S31508000D00801B8442F0D2F7E7DA68920644BF2022B5
S31508000D10DA60DB68DB0604D4044BD86810F00400FC
S31508000D2002D0FFF7A3FF012070BD00BF00200240DC
S31508000D302DE9F84F214C1F46237E012B054689468F
S31508000D40164637D001234CF250302376FFF7C6FFFC
S31508000D5060BB012D03D0022D0CBF022504254FF0E0
S31508000D600008DFF85CB0C2464FEA0812304639463A
S31508000D7000F0B6FFC4F81CA0DBF8103080B243F0D0
S31508000D800103CBF8103029F818004CF25030FFF761
S31508000D90A5FFDBF8103023F00103CBF8103028B993
S31508000DA008F101085FFA88F39D42DDD8002323760F
S31508000DB0BDE8F88F0220BDE8F88F00BF00060020C6
S31508000DC000200240B0F1904F08D1244B9A6A42F4B1
S31508000DD000329A629A6A22F400323AE0204B98422C
S31508000DE00BD103F1784303F503339A6A42F4802260
S31508000DF09A629A6A22F480222BE01A4B98420BD107
S31508000E0003F1784303F502339A6A42F400229A62A0
S31508000E109A6A22F400221CE0134B98420BD103F184
S31508000E20784303F501339A6A42F480129A629A6A01
S31508000E3022F480120DE00D4B98420DD103F1784350
S31508000E4003F5FE339A6A42F480029A629A6A22F499
S31508000E5080029A6201207047002070470010024005
S31508000E600004004800080048000C00480014004828
S31508000E702DE9F0430C6894FAA4F44FF00109B4FA8A
S31508000E8084F403250F260A6832FA04F300F08680F4
S31508000E9009FA04F313407FD0D0F800C093FAA3F2FE
S31508000EA0B2FA82F293FAA3FE4F68BEFA8EFE520099
S31508000EB005FA02F24FEA4E0E2CEA020207FA0EFE75
S31508000EC042EA0E0202604A68013A012A16D8D0F8A8
S31508000ED008C093FAA3F2B2FA82F293FAA3FE8F68D5
S31508000EE0BEFA8EFE520005FA02F24FEA4E0E2CEAC0
S31508000EF0020207FA0EFE42EA0E028260D0F80CC021
S31508000F0093FAA3F2B2FA82F293FAA3FE0F69BEFA33
S31508000F108EFE520005FA02F24FEA4E0E2CEA020243
S31508000F2007FA0EFE42EA0E02C2604A68022A33D166
S31508000F3093FAA3F2B2FA82F2072AD1F814E016DC81
S31508000F40D0F8208093FAA3FCBCFA8CFC93FAA3F29F
S31508000F50B2FA82F24FEA8C0306FA03F3920028EA01
S31508000F6003080EFA02F348EA0303036214E0D0F812
S31508000F7024C01B0A93FAA3F2B2FA82F293FAA3F3F5
S31508000F80B3FA83F3920006FA02F29B002CEA0202F5
S31508000F900EFA03F313434362013474E74B68013BCB
S31508000FA0012B06D8436823EA0204CB68534323433C
S31508000FB043600120BDE8F083064B0022DA61064B48
S31508000FC01A6942F004021A611A6942F040021A616B
S31508000FD0704700BF0006002000200240064B002292
S31508000FE0DA61064B1A6942F002021A6158611A69F7
S31508000FF042F040021A6170470006002000200240B5
S315080010002DE9F041234D2B7E012B074688463ED01D
S3150800101001242C760368A3424CF2503010D1FFF716
S315080010205DFE08B101202EE0FFF7C6FF4CF25030F6
S31508001030FFF754FE184A136923F00403136122E0EC
S31508001040FFF74CFE0028EDD14FF0FF33C8F800300B
S3150800105020467E68104CBA687B6803EBC2239E4222
S3150800106011D23046FFF7BAFF4CF25030FFF736FE82
S31508001070236923F00203236110B1C8F8006002E077
S3150800108006F50066E7E700232B76BDE8F081022027
S31508001090BDE8F0810006002000200240074AD36818
S315080010A023F4E0631B041B0C43F0BF63000243F404
S315080010B0003300F4E0600343D360704700ED00E0BE
S315080010C030B5174BDB68C3F30223C3F107041D1DB4
S315080010D0042C28BF0424062D4FF0010505FA04F454
S315080010E004F1FF348CBF033B00230C409C4005FAF7
S315080010F003F3013B1A40002842EA04024FEA0212AF
S31508001100AFBF00F1604000F00F00064BD2B2A5BF9A
S3150800111000F56140D2B21A5480F8002330BD00BFF2
S3150800112000ED00E014ED00E00138B0F1807F0AD24E
S31508001130064B074A5860F02182F823100020072240
S3150800114098601A6070470120704700BF10E000E001
S3150800115000ED00E0034B044A5B68C3F30313D35C5A
S31508001160D8407047001002409B1D0008034B044AF4
S315080011705B68C3F30223D35CD84070470010024073
S31508001180AB1D0008034B044A5B68C3F3C223D35C58
S31508001190D840704700100240AB1D000810B50E4A33
S315080011A00E4B50680E4900F48030002818BF1946C7
S315080011B0D06A52684FF4701393FAA3F3B3FA83F420
S315080011C002F47013E340023300F00F000130B1FB64
S315080011D0F0F0584310BD00BF0010024000127A001C
S315080011E000093D00044B5B6803F00C03082B01D192
S315080011F0FFF7D4BF014870470010024000127A007A
S3150800120010B50446FFF7EEFF2060FFF7A3FF606006
S31508001210FFF7ACFFA0606068FFF7B4FFE06010BDA1
S3150800122008B520BB134A136B03F00303022B0ED039
S31508001230032B05D0012B12D1BDE80840FFF7D2BF1A
S3150800124013680D4813F0020F08BF002008BD136A83
S3150800125013F0020F0CBF00204FF4004008BDFFF743
S31508001260C1FFFFF777FFBDE80840FFF77FBF002003
S3150800127008BD00BF0010024000127A0010B5074BE7
S315080012804FF0FF3200241A611C61DA60DC609A6252
S315080012909C62FFF707F9204610BD00BF0010024008
S315080012A010B5084B044618684FF47A73B0FBF3F090
S315080012B0FFF73AFF002221464FF0FF30FFF700FF05
S315080012C0002010BD0000002008B5074A136843F047
S315080012D0100313600320FFF7E1FE0020FFF7E0FF8D
S315080012E0FFF774F8002008BD00200240034BFE22D9
S315080012F0DA7002221871A3F844207047940000207F
S31508001300054B00221A709A6483F84320A3F84420F8
S315080013109A705A70704700BF94000020024B1878E4
S31508001320003018BF0120704794000020024B0022AD
S3150800133083F84320704700BF94000020F8B503786F
S31508001340814CFF2B054619D100220125E370102395
S31508001350237162706271257000F050F9A07100F077
S315080013603FF9E07100F03CF90823000A2072657223
S31508001370A572A4F8443000F021FACEE02678012EB2
S3150800138040F0E080F32B53D01ED8CF2B00F0B98065
S3150800139005D8C92B7FD0CC2B00F0BA80BAE0D12B68
S315080013A000F0A980C0F08980D22B40F0B3800025D8
S315080013B0FF23E3702571657100F020F9E571A071CE
S315080013C025726572072393E0FA2B46D00AD8F52BC7
S315080013D011D019D3F62B40F09D80FF23E3704368A4
S315080013E0A36492E0FD2B47D0FE2B50D0FC2B40F097
S315080013F0918000208FE000F001F96A78904201DCC4
S31508001400222088E0A16C07E000F0F8F86B78984293
S31508001410F6DD6968A1646A78201D00F007FAFF23E3
S31508001420E3706B78A26C1344A3646B7801335FE0B6
S31508001430FF23E370A26C4168002311448A4204D05A
S3150800144012F8010B0344DBB2F8E7C4F807300123AE
S31508001450237100236371A3710CE0FF23E3703B4BF8
S31508001460A3640722002323716371A371E2712372B7
S315080014706372A37208233BE0FF23E370627862710C
S3150800148000232371A371E3712372062330E000233E
S315080014902370637037E0A76C00F0B0F86A1C411E31
S315080014A0384600F08DF998B3FF23E37000F0A6F8EC
S315080014B0A36C01381844A06427E000F09FF86B7805
S315080014C0013898429CDDFF23E370A4F844606978EC
S315080014D019B900F07DF900BB1AE0AA1CA06C1A4ED7
S315080014E000F06EF9A0B16B78B26C1344B36414E0E3
S315080014F0A4F8443011E04168A06C00F063F910B913
S3150800150006E000F071F9FF23E370A4F8446004E0F4
S31508001510312000E02020FFF7E9FE94F84330012B44
S3150800152002D11020FFF7E2FEB4F94410064800295C
S3150800153008DD012380F8433089B20330BDE8F8405E
S3150800154000F036B8F8BD00BF94000020B31D0008AF
S3150800155010B5064CFFF7D4FE00F0E6FA0123237017
S3150800156000F0B2F80023237010BD00BF040000206D
S3150800157008B50C4800F058FB012804D10A4B18702E
S315080015800848FFF7DBFE074800F0D4F8012807D122
S31508001590054B044800221A70BDE80840FFF7CEBE86
S315080015A008BD00BFE00000200400002070470000CE
S315080015B070B50A4B1A78012A06460D461C4602D112
S315080015C0C9B200F011FB23781BB9E9B2304600F026
S315080015D095F8BDE87040FFF7A9BE00BF04000020DB
S315080015E0044B1B78013BDBB2022B9ABF024AD05C44
S315080015F04020704704000020BB1D0008FFF7F0BF1D
S31508001600FFF78CBE08B500F0ECF800F015F800F00E
S315080016102DFB00F0D3F8FFF79BFFBDE8084000F06C
S315080016202FB808B500F00AF800F036FBFFF7A0FF60
S31508001630BDE8084000F008B8FEF761BFFEF762BFD4
S3150800164008B5FFF7FBFFFCE710B5FFF7D9FF012840
S3150800165011D0094C2378012B0DD100F02BFB074B39
S315080016601B6803F5FA73984205D300232370BDE877
S31508001670104000F0B9B810BD200100202401002058
S3150800168008B5054B01221A7000F014FB034B1860CD
S31508001690BDE80840FFF7D8BF20010020240100203C
S315080016A038B5044600F006FB064BA4B21C85451D5A
S315080016B01C46E3691B0603D400F0FCFA8542F8D2FF
S315080016C038BD00BF0044004010B50B4C88B04FF43D
S315080016D0614301930C22002301A920460293039338
S315080016E00493069307930592FEF774FF236843F065
S315080016F00103236008B010BD00440040402970B5BE
S3150800170006460C4603D96D210948FFF799FF20467E
S31508001710FFF7C6FF3546A4B2AB1B9BB29C4206D95F
S31508001720FFF78CFF15F8010BFFF7BAFFF4E770BD5A
S31508001730BE1D000870B51C4D1C4A2C789CB9D3698F
S315080017409B0601D400242DE0938C194ADBB2137052
S31508001750002BF7D000F0AEFA164B1860164B1C702B
S3150800176001232B701EE0D46914F0200412D0124C09
S315080017700F492378968CCA18013356700A78DBB25B
S315080017809A422370DED1013100F050F800232B7005
S31508001790012407E000F08EFA064B1B686433984272
S315080017A0D0D92C70204670BD6E0100200044004040
S315080017B02C010020280100206D01002000F0E4B86B
S315080017C000F0E4B800F008B900F068B900F0A8B96C
S315080017D008B500F03FF918B1BDE8084000F086B931
S315080017E008BD00F078BA000010B5FFF7EDFFC8B1E4
S315080017F0FEF77CFEB0B1FFF7D9FE00F047FAFFF717
S315080018003DFDFFF7E3FF084B20F0604020F07F0026
S315080018109860FFF7DBFF446800F05FFA2346BDE8EF
S315080018201040184710BD00BF00ED00E0013A70B542
S315080018304D1E5618441AB54205D015F8013F635592
S31508001840FFF7FCFEF7E770BD2DE9F8430646FFF7FC
S3150800185029FA0024251DD6F80080775904EB0809D3
S31508001860FFF7ECFE3A46002349460220FFF760FAE6
S3150800187048B954F808309F4207D1B5F5007F2C4681
S31508001880E8D1012402E0002400E00446FFF71CFA30
S315080018902046BDE8F883000038B5114B9842044647
S315080018A00D4606D00F4A914205D0FFF7CDFF18B96D
S315080018B011E00D4C00E01C46C5F308035BB923682C
S315080018C09D420AD020464FF4007240F8045B294630
S315080018D0FFF7ACFF01E0002038BD204638BD00BF49
S315080018E07001002000200008740300202DE9F84349
S315080018F09846036821F4FF76013304460D461746D9
S3150800190026F0010606D140F8046B4FF40072314602
S31508001910FFF78CFF23689E4208D020463146FFF722
S31508001920BBFF044610B90020BDE8F8832368ED1A0A
S3150800193025440435B94606F50076FFF77FFE231DD4
S31508001940EB1AB3F5007F07D320463146FFF7A4FF0D
S3150800195004460028E7D0051D19F8013B05F8013BA8
S31508001960C9EB0803DF42E8D10120BDE8F88300008F
S31508001970034A4FF0FF331360024A1360704700BFF3
S315080019807403002070010020FFF7F2BF0B460D49D3
S31508001990884210B412D9591E0B4C0144A1420DD8E5
S315080019A020F4FF71094C21F00101A14201465DF8BE
S315080019B0044B0CBF06480748FFF798BF00205DF8A0
S315080019C0044B7047FF1F0008FFFF000800200008AF
S315080019D0700100207403002030B5024622F4FF632C
S315080019E01A4C85B023F007030020A34200902AD999
S315080019F04C1E174D1444AC4225D81144C91AC1F3DC
S31508001A00CF25C1F30A0109B10135ADB2002402930D
S31508001A10012301940393FFF745F9A3B29D420CD91C
S31508001A20FFF70CFE694601A8FFF7EAFA013430B958
S31508001A30029B03F500630293EFE7012400E000240C
S31508001A40FFF742F9204605B030BD00BFFF1F00086A
S31508001A50FFFF000807B50F4B1A68013215D09A68C0
S31508001A6059680D481144DA6811441A6911445A69CB
S31508001A7011449A691144DA698B1802AA5B4242F842
S31508001A80043D0421FFF782FF00E0012003B05DF862
S31508001A9004FB00BF70010020882100080D4B1A685E
S31508001AA004331B6813440C4A126813440B4A126821
S31508001AB013440B4A116804320B4412681A44094B42
S31508001AC01B681344084A1268D3420CBF0120002041
S31508001AD0704700BF00200008082000080C200008F6
S31508001AE010200008182000088821000808B50A48B0
S31508001AF00368013305D109480368013306D101207B
S31508001B0008BDFFF7A1FE0028F5D108BDFFF79CFE2A
S31508001B10003018BF012008BD7001002074030020A2
S31508001B200048704700200008F0B5294C8BB000200B
S31508001B304FF4FA754FF4FA472218035D5678991947
S31508001B4001FB055197FBF1F25143B1F5FA4F04D168
S31508001B5092B2511EB1F5806F09D302302428EBD119
S31508001B60AA211C48FFF76CFD00231E461A461A4C8C
S31508001B701A4921601A4921631A496163591E731E5D
S31508001B80002509041B052046216163616260A56181
S31508001B90E56125626562A562E562A560E560FEF716
S31508001BA0EEFD4CF6E04201238DE824004FF6E07284
S31508001BB007930292089304220E2369462046059548
S31508001BC00695039204950993FEF764FD0BB0F0BDE4
S31508001BD0091E0008E41D0008B8050020006400403E
S31508001BE0780500209405002070B40E4B1A6B40F25D
S31508001BF0E17414601C6B0022A2601C6BE2601A6B15
S31508001C0004461161221AD5B2A94205D91E6B14F8E9
S31508001C10015B32441575F5E73221024870BCFEF7C0
S31508001C204DBE00BFB805002038B50F4C002205464A
S31508001C3011462046FEF724FFA0B9636B196840F2E7
S31508001C40676291420FD19B686BB9626B1069D9B212
S31508001C50884203F1010303D90A44127D6A54F4E762
S31508001C60012038BD002038BDB8050020054B0022EC
S31508001C704FF6FF111A60596005219A601960024BE8
S31508001C801A60704710E000E0FC050020014B0022B6
S31508001C901A60704710E000E0044B1B68DB0341BF85
S31508001CA0034A136801331360704700BF10E000E071
S31508001CB0FC05002008B5FFF7EFFF014B186808BDC3
S31508001CC0FC05002008B5FFF7E7FF014B186808BDBB
S31508001CD0FC050020704772B6704762B67047000070
S31508001CE0D0400B1CD1409C46203AD3401843524260
S31508001CF0634693401843704708B5074B044613B12B
S31508001D000021AFF30080054B1868836A03B1984732
S31508001D102046FEF75DFC00BF00000000301E0008EC
S31508001D2070B50E4B0E4CE41AA41000251E46A542AB
S31508001D3004D056F8253098470135F8E700F01EF824
S31508001D40084C094BE41AA41000251E46A54204D0E7
S31508001D5056F8253098470135F8E770BD6800002029
S31508001D60680000206C00002068000020024403463A
S31508001D70934202D003F8011BFAE77047F8B500BF93
S31508001D80F8BC08BC9E467047F8B500BFF8BC08BC4E
S31508001D909E4670476D61696E2E6300000000000064
S31508001DA000000001020304060708090000000001FC
S31508001DB00203044F70656E424C54000800002E2E34
S31508001DC02F2E2E2F2E2E2F536F757263652F41528D
S31508001DD04D434D345F53544D333246332F7561723C
S31508001DE0742E63002E2E2F2E2E2F2E2E2F536F7508
S31508001DF07263652F41524D434D345F53544D333210
S31508001E0046332F63616E2E6300050206020603073A
S31508001E10030803090309040A040B040C040C050D42
S31508001E20050E050F050F061006100710080000001E
S30D08001E30080000200000000074
S30D08001E38ACE3FF7F0100000086
S31508001E4000127A00040000000000000000000000F4
S31508001E500000000000000000000000000000000074
S31508001E600000000000000000000000000000000064
S31508001E700000000000000000000000000000000054
S31508001E800000000000000000000000000000000044
S31508001E900000000000000000000000000000000034
S31508001EA00000000000000000AD01000889010008DC
S70508000000F2
